:020000040000FA
:10000000640001218613E3201322F72083168E1843
:1000100012288E148312403084202830B30096209A
:10002000B30B0F2883122F308420952095200E21AA
:1000300095200E213A08B6003B08B7008617952098
:100040000E213A08B8003B08B900861395200E210E
:1000500083164F30860083128F200608F300831624
:10006000403086008312731C4128F31C4828731DFE
:100070005228F31D51288613441C61284410232262
:10008000612844140A30F107031C6128F00A612832
:100090004414F630F107031C4E28F00AFF30F00735
:1000A00061288617F7200E21F5200B1D5A280030F5
:1000B00084202828A4013A08A3003B08A200262196
:1000C0002828F72095200E213A08031969280B1DCE
:1000D0006C28003084202828C201EA21E821061F6C
:1000E0007928CF21C208031D81281D3084202F21AB
:1000F0002828D321C208031D8128263084206421AA
:10010000282800308420282883169B001C141A08F5
:10011000831203190800A12083169B0A8628FD304C
:10012000F4006630F5009A28962096207E30F40080
:100130002030F500F50F9A28F40F9A2800340F3973
:10014000303EC003031DA728C100FE2041088616CB
:10015000B500350EAC203508F200721C86117218FD
:100160008615F21C0611F2180615721D86107219FA
:100170008614F21D0610F219061406160000061267
:100180004230F400F40BC22800341830B300BC0134
:10019000BD01BE01BF013C3084000430B4003330E7
:1001A00080078019F039801B0F398002840AB40B54
:1001B000CF28A20DA30DA40DBF0DBE0DBD0DBC0D0E
:1001C000B30BCB2808009620861206120330AC2011
:1001D00096200330AC200330AC200230AC200C3031
:1001E000FF202830FF200630FF200130FA28093098
:1001F000C0000230FC208F288612A828C030FC20C6
:10020000C02806309F00831600309F0037308100E1
:10021000F730850040308600831208000B11810101
:10022000BA01BB018316E73085009620F7308500C0
:1002300083120108BA00831601160000011283120E
:10024000BB0301083A0603191B290800C5209521A4
:10025000972199219B219D219F21A121A329430819
:10026000A1203C080F3903193B299F2099219B218C
:1002700093219D214E293D0E0F39031945299F20B9
:100280009B2193219D219F214E293D080F39031960
:1002900050299F2093219D219F21A1211130842845
:1002A0003E0E0F39031D5D292030A1203E080F3975
:1002B000031D5E292030A1205F299D219F21A121BE
:1002C0009321A321143084284308A1203C080F392E
:1002D000031970299F20992193219B219D21792920
:1002E0003D0E0F3903197B299F2093219B219D21CE
:1002F0009F21173084283D080F39031985299F2035
:100300009D219F219321A12191293E0E0F39031D8B
:100310008C292030A1208D299D219F219321A1216D
:10032000A3211A3084282E30A1283C0E9F283C0897
:100330009F283D0E9F283D089F283E0E9F283E087F
:100340009F283F0E9F283F089F28BE23AA294623A7
:10035000AA29F622C2043008A9003108AA003208EE
:10036000AB0008002908B0002A08B1002B08B20031
:100370002308A9002408AA002508AB0008002308C8
:10038000A9062906A906A3002408AA062A06AA0681
:10039000A4002508AB062B06AB06A5000800A72184
:1003A0000022A921DE29A921F221A9210022BF21B1
:1003B000A7210222B221A921BF21A721A41FE2293E
:1003C0002D30E3292030C300A4139A22C204C5288B
:1003D0000622EB2904220222A721B221A921FA2117
:1003E000BF21A529B221B830A5006030A400FA30A1
:1003F000A3000800B221A501A401A30101300F2A26
:100400007030072A3630072A3830072A3A308400FD
:10041000B221A501A4010008A300840A0008A200DB
:100420005922C2040800831651309B0083121E22F9
:10043000F0001C22F100080083169B0A83161C148E
:100440001A0883120800831651309B0070082D2271
:1004500071082C22831208009B0A9A001C15553043
:100460009D00AA309D009C149C18342A83128C1382
:1004700083160800AF012408031D442A2308A400A2
:100480000319542AA301AF152F08A502031D031C4D
:10049000B22B0310A41B512AA30DA40DA50B4A2AAD
:1004A000B22BA61FA4130034A401A301A201A5012D
:1004B00000349630A500A601A41F672AA209A3094B
:1004C000A409A20A0319A30A0319A40AA617AF01D3
:1004D0002408031D7C2A2308A4002208A300A201EB
:1004E000AF152408031D7C2A2308A400A301AF1123
:1004F0002F1624080319542A2F08A502031D031CD4
:10050000B22B0310A41B8A2AA20DA30DA40DA50BC8
:10051000822AB22B271B231C512AA21F512AA30A6D
:100520000319A40A031D512AA40CA30CA50A03193C
:100530003C2B512AA2012508031900342408A600E7
:10054000A4179630A502A51FEA2AA509A50A083016
:100550002502031CC62AA500A20D2308A200240818
:10056000A300A40108302502031CC62AA500A20D81
:100570002308A200A30108302502031CC62AA500F7
:10058000A20DA2012508031D0310CF2A2508031977
:10059000CF2A0310A40CA30CA20CA50BC92A271B5D
:1005A000221CDB2A031CDB2AA20A0319A30A031953
:1005B000A40AA41BEA2AA61F0034A409A309A209BD
:1005C000A20A0319A30A0319A40A0034A401A3016F
:1005D000A20100342714A71FFF34A401A61FFF3077
:1005E000A400A300A200A60DA40CFF342508031D3F
:1005F0002B080319542A24082A06A6002B08A5074D
:100600007E30031C072BA50203183C2B0A2BA502E6
:10061000031CB22B2408A2002308A100A217AA17CA
:100620000310A401A3011030AF00211C1D2B2908C9
:10063000A3072A0803182A0FA407A40CA30CA20CD2
:10064000A10C0310AF0B152BA41B2A2BA20DA30D7D
:10065000A40DA503271B231C392BA21F392BA30A8A
:100660000319A40A031D392BA40CA30CA50A031912
:100670003C2BA61FA4130034A714A71FFF34FF3080
:10068000A500A400A300A60DA40CFF342B08031999
:10069000BC2B25080319542A24082A06A600A417EF
:1006A000AA17AF012408A2002308A1002908A1026B
:1006B0002A08031C2A0FA202A201A101031C662B17
:1006C0000310A40CA30CA20C0130AF002B08A50250
:1006D000031C702B7E302F07A50703183C2B752BAE
:1006E0007E302F07A507031CB22B1030AE00A10DE2
:1006F000A20DA30DA40DAF0D2908A3022A08031C07
:100700002A0FA4022A0DAF042F1C882B21148F2B33
:100710002908A3072A0803182A0AA4072110AE0BE8
:10072000772B271B211CAB2B0310A30DA40DAF0DA2
:100730002908A3022A08031C2A0FA4022A0D2F0449
:100740000139A1070318A20A031DAB2BA20CA10CAF
:10075000A50A03193C2BA61FA2132208A4002108F6
:10076000A30000342715A71FFF340130A500A40102
:10077000A301A60DA40CFF34A715FF348030AA06F0
:1007800024082A06AF00A201A80125082B02031C99
:10079000DB2B2B08A0002508AB002008A5002A08A9
:1007A000A0002408AA002008A4002908A00023080B
:1007B000A9002008A3002B08031900342408A60070
:1007C000A417AA172B082502AB000319012C083027
:1007D0002B02031CF82BAB002908A8002A08A9004B
:1007E000AA0108302B02031CF82B2608A4000034B1
:1007F0002B080319012C0310AA0CA90CA80CAB0B95
:10080000FB2BAF1F0B2CA809A909AA09A80A0319D9
:10081000A90A0319AA0A2808A20729080318290FF8
:10082000A3072A0803182A0FA407AF1B1F2C031CB9
:100830008A2AA40CA30CA20CA50F8A2A3C2B03180D
:10084000672AA209A309A409A20A0319A30A031982
:08085000A40A8030A6063A2A32
:02400E00623F0F
:10420000200054006900640061006B002000200061
:1042100054006500720075006B007500720021008B
:1042200000006E00460000007000460000006D00B7
:1042300048000000750048000000200043002000F6
:104240003D002000200020002000000020004C0045
:1042500020003D002000200020002000000053002E
:1042600065007400740069006E00670021002E0074
:10427000740075006E006700670075002E00000076
:104280004C00430020004D00450054004500520002
:104290002D002D006F004F004F006F002D002D00EE
:0642A000000027001000E1
:00000001FF
